:020000040000FA
:060000008BEF1AF0120064
:062000008BEF1AF0120044
:06200800A4EF17F0120026
:0620180099EF18F0120020
:06202A0002003135000048
:1020300097000000040000002E3500009E00000004
:042040000300000099
:0C204400D9CFE6FFE1CFD9FF020EE12664
:10205000949C8B8C93869D6AA06A9F6AA26AF26A9E
:10206000F16AF06AD08E0B0EC16EC40EB56E230EEF
:10207000B46E929AF90EB16E9484040EBD6E9D8476
:102080009F840A0EBA6EB80EBB6E0B0EBC6EA0809B
:10209000A280F28EDF6A090EDF5C0AE2DF50EA6A94
:1020A000820FE96E000EEA227F0EEF6EDF2AF3D771
:1020B000DF6A070EDF5C0AE2DF50EA6A680FE96E4A
:1020C000000EEA22DFCFEFFFDF2AF3D7DF6A080E28
:1020D000DF5C0AE2DF50EA6A6F0FE96E000EEA2267
:1020E000DFCFEFFFDF2AF3D7010EDB6ADBCFF3FF91
:1020F000DB2AF350E66E93DAE55200093AE1DF6A33
:10210000070EDF5C14E2010EDBCFF3FFDB2AF35096
:10211000E66E85DAE552E66EDF50EA6A680FE96E30
:10212000000EEA22E552E750EF6EDF2AE9D7DF6AB8
:10213000080EDF5C14E2010EDBCFF3FFDB2AF35065
:10214000E66E6DDAE552E66EDF50EA6A6F0FE96E11
:10215000000EEA22E552E750EF6EDF2AE9D7010EC2
:10216000DBCFF3FFDB2AF350E66E59DAE5520001CC
:10217000776F020EE15C02E2E16AE552E16EE55240
:10218000E7CFD9FF1200D9CFE6FFE1CFD9FF020E8A
:10219000E1261FDA060E0001935D03E36D50020B8A
:1021A00001E00DD10001975101E109D104010C5169
:1021B000800B01E004D1DF6A070EDF5C4EE2DF50E6
:1021C000EA6A680FE96E000EEA22EFCF18F0090EF6
:1021D000185C35E2DF50EA6A680FE96E000EEA2209
:1021E000EF50EA6A820FE96E000EEA22010EEFCF8D
:1021F000DBFFDB50FF081FE0DF50EA6A680FE96E83
:10220000000EEA22EF50186E010E185204E0E84664
:10221000FE0B1806FCE1000177150CE0010EDB5007
:10222000186E196AFE0ED8801856000E1956010E47
:1022300018C0DBFF03D0DE527F0EDD6E03D0DE520E
:102240007F0EDD6EDF50EA6A600FE96E000EEA2253
:10225000010EDBCFEFFFDF2AAFD7DF6A080EDF5CAE
:1022600001E39ED0010EDF5206E0DFCFF3FFE84628
:10227000FE0BF306FCE100019E1502E1000E01D009
:10228000010EE76E010EE7CFDBFFDF5206E0DFCF86
:10229000F3FFE846FE0BF306FCE1E81C00019E1785
:1022A000DF50EA6A6F0FE96E000EEA22EFCF18F0F6
:1022B000090E185C65E2DF50EA6A6F0FE96E000EE6
:1022C000EA22EF50EA6A820FE96E000EEA22EF502E
:1022D000FF0853E0DF50EA6A6F0FE96E000EEA2252
:1022E000EF50EA6A820FE96E000EEA22EFCF18F093
:1022F000750E185C19E2DF50EA6A6F0FE96E000E86
:10230000EA22EF50186E010E185204E0E846FE0B68
:102310001806FCE10001771502E1000E01D0010E64
:10232000E76E010EE7CFDBFFDF50EA6A6F0FE96E61
:10233000000EEA22EF50EA6A820FE96E000EEA22EE
:10234000EF50890819E2DF50EA6A6F0FE96E000E5C
:10235000EA22EF50186E010E185204E0E846FE0B18
:102360001806FCE10001771502E1010E01D0000E14
:10237000E76E010EE7CFDBFF02D0010EDB6A02D071
:10238000010EDB6A010EDB50DF5206E0DFCFF3FF08
:10239000E846FE0BF306FCE100019E13DF2A5ED740
:1023A0009EC067F0080EE66E600EE66E000EE66EEA
:1023B00029EC17F0E552E552E5520001976B020E49
:1023C000E15C02E2E16AE552E16EE552E7CFD9FF56
:1023D0001200D9CFE6FFE1CFD9FFE6520401135135
:1023E000030A07E0010A01E009D0125101E001D01F
:1023F00000D0125101E002D02AD800D0E552E552B7
:10240000E7CFD9FF1200D9CFE6FFE1CFD9FFE652DF
:102410000001280E8D6F040E8E6F0001070E916F64
:10242000E552E552E7CFD9FF1200D9CFE6FFE1CF61
:10243000D9FFE6520001300E8D6F040E8E6F000141
:10244000030E916FE552E552E7CFD9FF1200D9CFC5
:10245000E6FFE1CFD9FF030EE126020E30C4DBFF19
:102460000401306BDB50090A01E1A0D0010A55E0FC
:102470000F0A50E0010A40E0030A30E0010A2AE0B6
:10248000070A19E0010A08E0030A01E098D0306960
:10249000010E316F326B93D031C4DFFF070EDF5C6A
:1024A00009E23069DF50EA6A680FE96E000EEA223D
:1024B000EFCF31F484D031C4DFFF080EDF5C09E2D6
:1024C0003069DF50EA6A6F0FE96E000EEA22EFCF43
:1024D00031F475D0306977C031F471D031C4DFFF89
:1024E000070EDF5C08E2DF50EA6A680FE96E000E53
:1024F000EA2232C4EFFF63D031C4DFFF080EDF5C95
:1025000008E2DF50EA6A6F0FE96E000EEA2232C479
:10251000EFFF55D032C477F052D0DF6AE66ADF5061
:10252000DF2AE66E90D8E552E552010EDB6A070E0F
:10253000F36E010EDBCFF4FFF350F45C12E2010EF8
:10254000DB50EA6A680FE96E000EEA22EF50E66E91
:10255000DF50DF2AE66E77D8E552E552010EDB2A1E
:10256000E6D7010EDB6A080EF36E010EDBCFF4FF37
:10257000F350F45C12E2010EDB50EA6A6F0FE96E71
:10258000000EEA22EF50E66EDF50DF2AE66E5BD8DF
:10259000E552E552010EDB2AE6D777C0E6FFDF50B1
:1025A000DF2AE66E50D8E552E55209D0680E315D5B
:1025B00005E1620E325D02E120EC1AF000D0030E5C
:1025C000E15C02E2E16AE552E16EE552E7CFD9FF54
:1025D000120000019F51A01104E1400E9F6F9C0E5C
:1025E000A06F9F07000EA05B6DA209D0E80E9F5D53
:1025F000030EA05902E28B8C01D08B9C0FD0060EEB
:102600000001935D02E18B8C09D00001100E9F5DEB
:10261000270EA05902E28B9C01D08B8C1200D9CFDF
:10262000E6FFE1CFD9FFE652FE0EDB50A96EA69E73
:10263000A69CA680A850DF6EDF5000D0E552E55280
:10264000E7CFD9FF1200D9CFE6FFE1CFD9FFFE0EC9
:10265000DB50A96EFD0EDB50A86EA69EA69CA6843C
:10266000F29E550EA76EAA0EA76EA682F28EA1A8A4
:0E267000FED7A198A694E552E7CFD9FF12003D
:02267E00040155
:102680001051600BE842E842E842E842E8420009A3
:1026900001E055D01151070A51E00B0A4FE0070A3B
:1026A00040E0010A2CE00B0A28E0020A26E0030AB7
:1026B00022E0080A12E0010A0EE00F0A0AE0030A0B
:1026C00001E03CD00001010E8C6F0001040E936FFD
:1026D00036D036D834D090D832D00001010E8C6F6D
:1026E0000001950E8D6F000E8E6F00019493000116
:1026F000010E916F24D0A8D822D0F5D820D00001A7
:10270000010E8C6F0401145100018D6F8E6B960EBB
:102710008D27000E8E23000194930001010E916F0E
:102720000ED00001010E8C6F04011451EA6A960F5D
:10273000E96E000EEA2212C4EFFF01D000D01200B1
:10274000800E0401105D57E11351030A34E0010AC1
:1027500010E0030A01E04DD00001010E8C6F000172
:10276000DE0E8D6F320E8E6F120E0001916F926B26
:1027700040D00001010E8C6F04011251F66EF76A11
:10278000D890F636F736960EF626330EF722090065
:10279000F5CF8DF00A00F5CF8EF0020E0001F76A3A
:1027A0008D25F66E8E51F7220900F5CF91F00A00C3
:1027B000F5CF92F01ED00001010E8C6F0401125172
:1027C000F66EF76AD890F636F7369A0EF626330E7E
:1027D000F7220900F5CF8DF00A00F5CF8EF08DC0FD
:1027E000F6FF8EC0F7FF0800F5500001916F926B65
:1027F00000D00001948312000001010E8C6F0F0EB7
:10280000E66E710EE66E0F0EE66E5AEC19F0E552AA
:10281000E552E552010EE66E960EE66E000EE66E8D
:102820005AEC19F0E552E552E55212C495F0040154
:10283000125104E10001050E936F05D00001060E50
:10284000936F14EC17F012000401186B196B04015C
:1028500010511F0B020A15E0030A0FE0010A01E004
:1028600034D00001010E8C6F02D0040118810001E8
:1028700094A102D00401188328D00001010E8C6FAE
:1028800024D00001010E8C6F040114510F0B080DB0
:10289000F350196A000F186E040E19221451800BA0
:1028A00001E0010E040DF350000118248F6F000E9B
:1028B0001920906F8FC0E9FF90C0EAFFEF50040B22
:1028C00003E00401010E186F00D000018C050AE13D
:1028D0000001180E8D6F040E8E6F0001949300019D
:1028E000020E916F12000401120510E110511F0B2E
:1028F00000090CE10001010E8C6F030E0401115D53
:1029000003E10001948102D000019491040112516D
:102910003AE110511F0B020836E114510F0B000968
:1029200032E00001010E8C6F040114510F0B080DF1
:10293000F350196A000F186E040E19221451800BFF
:1029400001E0010E040DF350000118248F6F000EFA
:102950001920906F030E0401115D07E1840E8FC0F2
:10296000E9FF90C0EAFFEF6E0ED014AF06D08FC023
:10297000E9FF90C0EAFFEF6A06D0880E8FC0E9FF3A
:0829800090C0EAFFEF6E1200A7
:082988006C5002E0000E01D0CA
:10299000010E00090BE0040100513C0BE842E84243
:1029A0000D0802E10CD801D040D808D06C5002E0EC
:1029B000000E01D0010E040901E04DD81200D9CF5C
:1029C000E6FFE1CFD9FFE65200018B6B8C6B916B78
:1029D000926B3FEC13F0DF6ADF50186E196A010E3C
:1029E000185C000E19581BE200018C5101E017D051
:1029F000F76ADF34FE0BF736F66EA00EF626330EBE
:102A0000F7220900F5CF18F00800F5CF19F004D02F
:102A100019C0FAFF1850F96EFBDFDF2ADDD7E3D8C3
:102A2000E552E552E7CFD9FF1200020E00018B5D9F
:102A300010E19CD8020E00018C5D02E1E9EC11F07E
:102A4000040100BD03D0C80E006F02D0880E006FD5
:102A500001D00FD91200040E0001935D0AE112C4E7
:102A60006EFF6E50000803E2050E936F02D0030E56
:102A7000936F00018B050AE10BD8040104BD03D05C
:102A8000C80E046F02D0880E046F01D0F2D8120075
:102A9000D9CFE6FFE1CFD9FF020EE1260001080EF3
:102AA000915D000E925905E291C0DEFF92C0DDFFFC
:102AB00003D0080EDE6EDD6A040104930491010E5A
:102AC000DB500413DFCF05F4000EDB500001915FF3
:102AD000010EDB50925B180E8F6F040E906F000199
:102AE00094A31ED0D9CFE9FFDACFEAFFEE50ED1064
:102AF00016E08DC0F6FF8EC0F7FF0800F5508FC0BE
:102B0000E9FF90C0EAFFEF6E00018F2B000E9023CB
:102B10008D2B8E23DF06010E01E2DB06E3D71CD0EE
:102B2000D9CFE9FFDACFEAFFEE50ED1015E08DC006
:102B3000E9FF8EC0EAFFEF508FC0E9FF90C0EAFFC7
:102B4000EF6E00018F2B000E90238D2B8E23DF065E
:102B5000010E01E2DB06E4D7020EE15C02E2E16A6B
:102B6000E552E16EE552E7CFD9FF1200D9CFE6FF7B
:102B7000E1CFD9FF020EE126030E04010015E76E36
:102B8000010EE7CFDBFF01C4DFFFDE50000191271C
:102B9000DD509223180E8D6F040E8E6FD9CFE9FF92
:102BA000DACFEAFFEE50ED1014E08DC0E9FF8EC0E1
:102BB000EAFFEF508FC0E9FF90C0EAFFEF6E8F2B66
:102BC000000E90238D2B8E23DF06010E01E2DB0623
:102BD000E5D7020EE15C02E2E16AE552E16EE55200
:102BE000E7CFD9FF120000018C510CE10401080E5F
:102BF000016F100E026F040E036F840E006F04014C
:102C0000046F35D0040110AF22D0000191510401AE
:102C1000165D000192510401175904E216C491F0A7
:102C200017C492F035DF0001010E8B6F0401080E0E
:102C3000016F100E026F040E036F800E006F04010F
:102C4000180E066F040E076FC80E046F10D0000137
:102C5000020E8B6F0401056BC80E046F0401080E91
:102C6000016F180E026F040E036FC80E006F6D988F
:102C7000120000018B6B0401080E016F100E026F31
:0E2C8000040E036F880E006F0401046B120037
:022C8E0004013F
:102C900010511F0B010801E079D0145101E076D0EA
:102CA000060E115D2EE11351230A28E0010A13E0FC
:102CB000030A01E024D00001020E8C6F000195058B
:102CC00005E10001020E8D6F330E8E6F090E0001BB
:102CD000916F926B14D00001020E8C6F000195056C
:102CE00005E100014E0E8D6F330E8E6F00019505CC
:102CF00004E1480E0001916F926B01D000D00001F9
:102D0000948304011051600BE842E842E842E84233
:102D1000E842010801E03AD011510B0A31E0080AFB
:102D200021E0090A19E0080A09E00B0A05E0080A8F
:102D300001E02CD02CD82AD055D828D00001020E82
:102D40008C6F00019B0E8D6F000E8E6F00019493AF
:102D50000001010E916F1AD00001020E8C6F13C496
:102D60009BF014D00001020E8C6F00019C0E8D6F41
:102D7000000E8E6F000194930001010E916F06D03A
:102D80000001020E8C6F12C49CF000D01200D9CF4B
:102D9000E6FFE1CFD9FFE65204011351030A11E027
:102DA000020A01E018D01251010A09E0010A01E00B
:102DB00007D00001020E8C6F03EC12F001D000D09E
:102DC0000AD0125101E006D00001020E8C6F15EC02
:102DD00012F000D000D000019493E552E552E7CF05
:102DE000D9FF120004011351030A10E0010A01E0A7
:102DF0001AD0125101E009D00001020E8C6F0001BF
:102E0000200E8F6F040E906F00D00DD0125101E094
:102E100009D00001020E8C6F0001300E8F6F040E7E
:102E2000906F00D000D0120000019D6B1E0E716EDD
:102E30000401080E096F200E0A6F040E0B6F880E36
:102E4000086F0401280E0E6F040E0F6F400E0C6FFA
:102E50001200D9CFE6FFE1CFD9FFE652FC0EDB50DE
:102E6000080805E2080EF36EFC0EF3CFDBFFDF6A05
:102E7000FC0EDB50DF5C19E2DF50E76EFD0EDBCFAE
:102E8000E9FFFE0EDBCFEAFFE750E926000EEA225B
:102E9000EF50E66EDF50EA6A280FE96E040EEA2270
:102EA000E552E750EF6EDF2AE3D7FC0EDBCF0DF4DF
:102EB000400E04010C170C7D880E0C13E552E552F0
:102EC000E7CFD9FF1200D9CFE6FFE1CFD9FF00014C
:102ED0009D6B040108BF31D0FC0EDBCF18F0095107
:102EE000D880185403E2FC0E09C4DBFF00019D6B7F
:102EF000FC0EDB509D5D19E29D51EA6A200FE96EE0
:102F0000040EEA22EF50E66E9D51E76EFD0EDBCF18
:102F1000E9FFFE0EDBCFEAFFE750E926000EEA22CA
:102F2000E552E750EF6E9D2BE3D70401080E096FC1
:102F3000400E0817087D880E081300019D5100D02F
:082F4000E552E7CFD9FF1200B2
:082F4800DACFE4FFE2CFDAFF6B
:102F5000E9CFE4FFEACFE4FFF6CFE4FFF7CFE4FFE9
:102F6000F3CFE4FFF4CFE4FFFACFE4FF00EE00F08C
:102F7000140EE80403E3EECFE4FFFBD7E652D9CF0B
:102F8000E6FFE1CFD9FF050EE1269EA46ED0BECFAD
:102F9000DEFFBFCFDDFFDECFBBFFDDCFBCFFC40E4A
:102FA000BB26090EBC22A190FF0E0001985D57E0E0
:102FB0009951DE5C146E9A51DD58156E020E14C0E4
:102FC000DBFF030E15C0DBFFD950020FE96EDACF2D
:102FD000EAFFE80ED880EE54030EED5431E2020E03
:102FE000DBCF14F0030EDBCF15F0E80E145E030EFA
:102FF000155A020E0F0B05E0D89015321432E80670
:10300000FBE1020E14C0DBFF030E15C0DBFFD9503D
:10301000020FE96EDACFEAFFFE0ED880EE54000E02
:10302000ED5407E2FE0EF36E020EF3CFDBFF030E4C
:10303000DB6A020EDB50E76E040EE7CFDBFF02D047
:10304000040EDB6A090E0001985D09E29851EA6AF4
:10305000820FE96E000EEA22040EDBCFEFFFDECF17
:1030600099F0DDCF9AF0982B9E94A1A03FD08A963C
:10307000B250DE6EDD6AB350166E176A086A010E32
:10308000096E16C00DF017C00EF054EC1AF006C011
:1030900014F007C015F0D9CFE9FFDACFEAFF1450DA
:1030A000EE261550ED22DECFBBFFDDCFBCFFC40EF8
:1030B000BB26090EBC2200019851000805E2090E4A
:1030C000985D02E2010E976FFF0E985D01E1986B2B
:1030D000090E985D09E29851982BEA6A820FE96E11
:1030E000000EEA22EF68F4D79869A190050EE15C22
:1030F00002E2E16AE552E16EE552E7CFD9FFE5521F
:1031000000EE13F0140EE80403E3E5CFEDFFFBD768
:10311000E5CFFAFFE5CFF4FFE5CFF3FFE5CFF7FF0B
:10312000E5CFF6FFE5CFEAFFE5CFE9FFE5CFDAFF30
:103130001100D8CFE4FFE0CFE4FFE46EDACFE4FF84
:10314000E2CFDAFFE652E552E5CFDAFFE550E5CF10
:08315000E0FFE5CFD8FF1000FD
:083158006DA60FD802D06DB680
:1031600013D80001930508E16DBA06D0686A696A50
:1031700069806988020E936F12006D6A696A6D86B4
:103180000001010E936F12006D6A696A0001936B72
:103190001200C4EF18F00001935101E13AD06850D9
:1031A000040B04E06950040B01E041D86DB231D04A
:1031B0006850010B04E06950010B01E059D86850D8
:1031C000100B04E06950100B01E024D86850400B4C
:1031D00004E06950400B01E040D86850200B04E047
:1031E0006950200B01E03BD86850020B04E06950A5
:1031F000020B01E03BD8030E0001935D01E209D010
:103200006850080B06E06950080B03E0C4EC14F0AA
:1032100068961200698468986D82A19AF290A08ADB
:10322000F2860300F2B007D8A09AF29612006D92CF
:10323000699468941200000194A10ED0F8DF6D84A7
:103240000001080EA16F070EA26FA107000EA25B7E
:10325000A151A211FAE16D941200689C120070A0B5
:1032600003D039EC16F07090689A12006892120040
:103270006A6A686A9F0E6B6E7B0E696E6E6A0F0ECD
:10328000E66E710EE66E0F0EE66E14D8E552E5524C
:10329000E552160E706E68A602D06896FCD76D983F
:1032A00039EC16F0000194910001956B0001030EBA
:1032B000936F1200D9CFE6FFE1CFD9FFFD0EDBCF30
:1032C000E9FFFE0EDBCFEAFFFC0EDB5004E0EE6A06
:0E32D000FC0EDB06F9D7E552E7CFD9FF12005E
:0232DE001201DB
:1032E0000002000000088117F4080100010200013B
:1032F00009022200010100A03209040000010301BB
:10330000020009210101000122480007058103088C
:10331000000A040309041E034700610064006700FB
:103320006500740050006100720061006400690073
:10333000730065001A0352002F00430020004A006A
:103340006F0079000000000000000000000005018F
:103350000904A1017508150026FE0005010901A157
:10336000000930093195028102C00932093309345C
:103370000935093695058102050919012908150045
:1033800025017501950881020905150026FF0075C4
:10339000089503B102C0F032F032123316333433E1
:0233A0008E2C71
:0E33A2002A0EF66E200EF76E000EF86E000179
:1033B0000900F5507D6F0900F5507E6F03E17D67D0
:1033C00001D03DD00900F550786F0900F550796FB4
:1033D0000900F5507A6F09000900F550E96E0900FF
:1033E000F550EA6E090009000900F5507B6F0900ED
:1033F000F5507C6F09000900F6CF7FF0F7CF80F021
:10340000F8CF81F078C0F6FF79C0F7FF7AC0F8FFF7
:1034100000017B5302E17C5307E00900F550EE6E9A
:103420007B07F8E27C07F9D77FC0F6FF80C0F7FF83
:1034300081C0F8FF00017D07000E7E5BBFD7120040
:10344000D9CFE6FFE1CFD9FF020EE126C9EC18F093
:10345000840EA66EFE0EF66E5F0EF76EF86AF56AC3
:103460000C00550EA76EAA0EA76EA682DE6ADD6A54
:10347000D9CFE9FFDACFEAFFEE06000EED5AEECF24
:1034800018F0EDCF19F01850191003E000000000FB
:10349000EFD7FF00020EE15C02E2E16AE552E16E65
:0834A000E552E7CFD9FF12004D
:0834A80008C012F008500D02EB
:1034B000F4CF07F0F3CF06F009500E02F4CF09F075
:1034C000F3CF08F00D02F3500726F4500822E86A03
:1034D000092212500E02F3500726F4500822E86A1F
:0434E0000922000CB1
:0C34E40005D810D8C3EC10F0FCD7120083
:1034F0000F0EC112140E6F6E0001936B0001946BDE
:103500000001956B22EF10F0ACEC18F06FBE02D00A
:06351000CBEC18F01200E4
:0A35160013EE00F023EE00F0F86A57
:0E352000019CD1EC19F072EC1AF0FDD71200EC
:02352E0000009B
:01353000009A
:0435310000FF000097
:020000040030CA
:0100000028D7
:010001000EF0
:0100020026D7
:010003001EDE
:010005008179
:010006008178
:010008000FE8
:01000900C036
:01000A000FE6
:01000B00E014
:01000C000FE4
:01000D0040B2
:0200000400F00A
:10000000000001020304050604FFFFFFFFFFFFFFDE
:0100100000EF
:00000001FF
